:1000000009298030A100FE30A7200130A7207530DB
:10001000A7003030BE28A101A117AF00AF08031D13
:100020001328030114280130AF020310A20CA20C04
:10003000A20CC0302205403EAF07FE30A7202F089B
:10004000A728A101A117AF00FE30A7202F08A728DD
:10005000A401AA00AB01A01124080319A0150530C2
:10006000A3002730A900103041200330A900E83058
:100070004120A90164304120A9010A3041202A0809
:100080004828A8002B08A7002A08A600D220260886
:10009000A600A3030319A011240803195228230260
:1000A000031859282608031DA011A0195928303E0D
:1000B000A7280800AD0006118611831606118611C7
:1000C0000F30860583122D08A01884283E30A70023
:1000D0008030BE203330AC0098201330A700883029
:1000E000BE2098206430BD2098206430BD2022308E
:1000F000AC009820283083200C30832006308320E9
:10010000A0142D0884282014AC00201C92288611ED
:10011000033C031C972897200530A700DC30BE2045
:10012000031408002014FE3C0319A5288615201C82
:10013000201006150F3086052C08F03986040611AC
:10014000AC0E201898283230BD202D080429A11BA0
:100150005A2883178001840AFF3E031DAA28042918
:10016000A901A800FF30A807031CA907031C042944
:100170000330A700DF30BE20B228A701E83EA6006A
:10018000A709FC30031CC728A6070318C428A60724
:100190000000A70FC4282618CD28A61CD1280000CF
:1001A000D1280800AB01AA011030AC00270DAA0D20
:1001B000AB0D2808AA022908031C290FAB0203185B
:1001C000E8282808AA0729080318290FAB070310F5
:1001D000A60DA70DAC0BD628260804291030B000B8
:1001E000A701A601AD0CAC0C031CFC282808A6072F
:1001F00029080318290FA707A70CA60CAB0CAA0CFB
:10020000B00BF2282A080429831383120313000079
:100210000800A00107309F00E03083168500FF3002
:1002200086008113831285018601203084006030AE
:10023000AA20A03084005030AA2020308400303022
:10024000A920C830B020012077305A205A205A20E7
:100250002E305A2070305A2069305A2063305A208C
:1002600062305A2061305A2073305A2069305A2047
:1002700063305A202E305A206E305A206C305A206B
:100280000B30A900B830B120012044305A2043304F
:100290005A2046305A2032305A2034305A204E30BC
:1002A0005A204C305A2041305A2020305A205A20AF
:1002B00056305A202D305A2032305A200730A900AB
:1002C000D030B12001204C305A2044305A205230D6
:1002D0005A2020305A2061305A2066305A2072301D
:1002E0005A2065305A2067305A2065305A206C30C9
:1002F0005A2065305A206E305A2086188529851F6D
:1003000083290514842905107D29012053305A20A2
:1003100069305A2067305A206E305A2061305A2096
:100320005A206C305A2020305A207A305A206F30B0
:100330005A2065305A206B305A2065305A206E3072
:100340005A20361405128316051283122A2AC30175
:100350003C03A500C90149082502031CC029E3216B
:10036000B61CBE294308A6004908A200A601A20A9D
:100370000314A60DA20BB9292608C304C90FAB2983
:10038000B2014308B100B20CB10CB20CB10CB20C0A
:10039000B10CB20CB10C0F30B2053208AD0031080F
:1003A000AC00A9010A30A800EE20B1002B08B20071
:1003B000B4014308B3000F30B3050030B405310871
:1003C0003307C3000800BA01B9010618F829013043
:1003D000B020B90A0319BA0A0B303A02031CF729F4
:1003E000031DF629B9303902031CF729C62CE5296B
:1003F0009B30B0200618B614061CB610361C142A02
:10040000AD014408AC00A9011830A800EE20B100ED
:100410002B08B2003208A7003108A600A9013A3023
:10042000A800D220BD001D2A03013619013EB618CE
:10043000013A03193611031D3615C40A851401301B
:10044000A900F430B1208510A901F030A8002808D7
:10045000B1200800BB01C4013612361ABD2ABA0108
:10046000B901061C442AB90A0319BA0A0130B0209E
:10047000AF303A02031C432A031D422AC930390215
:10048000031C432AC62C312ABA01B9010618762A60
:10049000B90A0319BA0A0A30B02036186A2A39088C
:1004A0000B3A3A04031D552A692A3908193A3A04C5
:1004B000031D5C2A8514692A39084B3A3A04031D46
:1004C000632A8510692A3908FA3A3A04031D692A11
:1004D000C62C752A11303A02031C752A031D742A92
:1004E00095303902031C752AC62C462A41303B023E
:1004F000031C7B2AC62CBB0A3A08031D832A6530DD
:100500003902031C842A3616361CBC2AAD013B086E
:10051000AC00A9011830A800EE20B1002B08B200F1
:100520003208A7003108A600A9014130A800D22056
:10053000BD008030A1008030212053305A20693026
:100540005A2067305A206E305A2061305A205A2083
:100550006C305A2020305A2067305A2065305A209B
:1005600076305A206F305A206E305A2064305A202C
:1005700065305A206E305A202D2A361CDF2A012081
:1005800049305A206E305A2069305A2074305A202F
:1005900069305A2061305A206C305A2069305A2014
:1005A00073305A2065305A2072305A2065305A20F4
:1005B0006E305A202E305A205A205A20492B1230A1
:1005C000BD000130A2003D080B20A101B61DF72A95
:1005D0003B3041020318EE2AC10AF62AC101173046
:1005E00045020318F52AC50AF62AC501FB2A420866
:1005F000C1004608C500051B0B2B4508031D032B36
:100600000C30C7000A2B0D304502031C0A2B0C309E
:100610004502C700102B4508C70020305A205A2039
:100620000A3047020318162B20305A208030A100D0
:10063000470828203A305A200230A40041082920D7
:10064000051B322B0C30450203182B2B61305A202E
:100650006D305A202F2B70305A206D305A201530B3
:10066000BD00342B1730BD00410803190130031DB4
:100670000301B5001E30410203190130031D0301BF
:100680003504B50001308618030135040319492BE0
:100690009E2C361E9C2CE3210130C9000F304902EC
:1006A0000318552BE321C90F4E2B3611B611E32148
:1006B000E321E321B61C5E2B05145F2B05101230DD
:1006C000C900143049020318682BE321C90F612BBC
:1006D000E3210730BC00A7214308C200E321361DF7
:1006E000722BB6150630BC00A7214308C600E321D3
:1006F000361D7B2BB6150630BC00A7214308BE0073
:100700000330BC00A7214308C8000530BC00A72166
:100710004308C0000830BC00A7214308BF00E32104
:10072000361D932BB615361C992BB619982B3610FF
:100730000120B6199B2C8030A100803021203E087A
:10074000282020305A2001304002031DB62B6A3089
:100750005A2061305A206E305A2075305A2061304C
:100760005A2072305A2069305A20752C02304002CB
:10077000031DCB2B66305A2065305A2062305A2038
:1007800072305A2075305A2061305A2072305A2007
:1007900069305A20752C03304002031DD92B6D306F
:1007A0005A2061305A205A2072305A2074305A2010
:1007B000752C04304002031DE82B61305A20703044
:1007C0005A2072305A2069305A206C305A20752CC9
:1007D00005304002031DF32B6D305A2065305A203E
:1007E00069305A20752C06304002031D002C6A30F7
:1007F0005A2075305A206E305A2069305A20752C94
:1008000007304002031D0D2C6A305A2075305A20E3
:100810006C305A2069305A20752C08304002031D74
:10082000222C61305A2075305A2067305A2075309A
:100830005A2073305A2074305A2075305A20733041
:100840005A20752C09304002031D392C73305A2070
:1008500065305A2070305A2074305A2065305A2042
:100860006D305A2062305A2065305A2072305A203A
:10087000752C0A304002031D4C2C6F305A206B300F
:100880005A2074305A206F305A2062305A20653016
:100890005A2072305A20752C0B304002031D612CF7
:1008A0006E305A206F305A2076305A2065305A20E8
:1008B0006D305A2062305A2065305A2072305A20EA
:1008C000752C0C304002031D752C64305A206530A5
:1008D0005A2063305A2065305A206D305A206230D9
:1008E0005A2065305A2072305A200130051B03010E
:1008F000B5000930400203190130031D030135051D
:1009000003198F2C20305A2027305A208030A10024
:100910000230A4003F08292020305A209B2C203090
:100920005A2032305A2030305A208030A100023014
:10093000A4003F0829209D2CC62C2A2A851FA52CFF
:100940000512831605128312A72C8316051683122F
:100950009B30B020410803190130031D0301B5008D
:1009600001308618030135040319B72C05158515C8
:1009700085140130A900F430B120051185118510CE
:100980000130A9004A30B120C40A4C2B0120473065
:100990005A2065305A205A206E305A2020305A2072
:1009A00073305A2069305A2067305A206E305A20EE
:1009B00061305A205A206C305A2020308400603038
:1009C000AA20A03084005030AA202030840030308B
:1009D000A9200618B616061CB61203010618013E19
:1009E000B61A013C031DFA2CB70A0319B80A0130E4
:1009F000B020ED2C0301B61A0130013A0319B612EA
:100A0000031DB61603010618013EB61A013C031D6C
:100A10000F2DB70A0319B80A0130B020022D033098
:100A20003802DE30031937020318DD2C36142A2A67
:02400E00503F21
:00000001FF
